:04000000AAEF02F071
:100018000180D8CF04F0E8CF05F0E0CF06F0D9CFC3
:1000280007F0DACF08F0F3CF09F0F4CF0AF0010EA9
:10003800F0A0000EF0A6000EE8A003D0026A022A83
:1000480001D0026A0250D8B451D080CF14F082CFC8
:100058000DF083CF13F084CF0FF081CF0EF00EA6F2
:1000680044D014A202D0118001D0119014AA02D059
:10007800118201D011920FA002D0118401D01194E5
:1000880014A002D0118601D0119614AE02D01188A6
:1000980001D0119813A602D0118A01D0119A0DAA85
:1000A80002D0118C01D0119C0FA402D0118E01D066
:1000B800119E1104D8A404D0010E0001756F15D04B
:1000C80000017551D8B406D0C00E1118D8B44B6AC7
:1000D800756B0BD0140E4B6008D04B508B0FD96E3C
:1000E800DA6A11507F0BDF6E4B2AF090010EF0A2F6
:1000F800000EF0A8000EE8A003D0026A022A01D080
:10010800026A0250D8B451D080CF14F082CF0DF0DB
:1001180083CF13F084CF0FF081CF0EF00EA644D01A
:1001280014A202D0118001D0119014AA02D0118219
:1001380001D011920FA002D0118401D0119414A003
:1001480002D0118601D0119614AE02D0118801D0C8
:10015800119813A602D0118A01D0119A0DAA02D0C3
:10016800118C01D0119C0FA402D0118E01D0119EC8
:100178001104D8A404D0010E0001746F15D0000139
:100188007451D8B406D0C00E1118D8B44A6A746B2A
:100198000BD0140E4A6008D04A50760FD96EDA6A2E
:1001A80011507F0BDF6E4A2AF092F2A0BFD1080EE1
:1001B800026E440EE82EFED7022EFCD700D080CF68
:1001C80014F082CF0DF083CF13F084CF0FF081CFDE
:1001D8000EF00E380F0B156E040E4918D8A458D01F
:1001E8000001704B712B410E705D060E7159D8A03D
:1001F80032D0716B000E706F0C6A0C50020D200E1D
:10020800F324D96E010EF420DA6E010EDB5004E1FE
:10021800330EDE5CD8A009D0400E0C24D96EDA6A01
:10022800010EDA22010EDF6E07D0400E0C24D96EC3
:10023800DA6A010EDA22DF6A0C50020D200EF3246E
:10024800D96E010EF420DA6EDE6ADD6A0C2A0F0E12
:100258000C64D3D76AD11550020D200EF324D96E41
:10026800010EF420DA6EDECF02F0DDCF03F0010ECE
:100278000226000E03221550020D200EF324D96E1B
:10028800010EF420DA6E02C0DEFF03C0DDFF4DD19F
:10029800030E4918D8A48BD014A002D0128E01D016
:1002A800129E14A202D0128001D0129014A402D07F
:1002B800128C01D0129C14A602D0128201D0129284
:1002C80014A802D0128A01D0129A14AA02D0128459
:1002D80001D012940FA002D0128801D012980EA259
:1002E80002D0128601D012960FA402D0108E01D02F
:1002F800109E14AE02D0108001D0109013A002D02E
:10030800108C01D0109C13A202D0108201D0109240
:1003180013A402D0108A01D0109A13A602D0108418
:1003280001D010940DAA02D0108801D010980EA404
:1003380002D0108601D01096060E156009D015500F
:100348003E0FD96EDA6A12C0DFFF1550300F1CD08D
:10035800060E1518D8A403D012C045F0E6D0070E33
:100368001518D8A403D012C046F0DFD0070E1564C4
:1003780010D00E0E15600DD015502F0FD96EDA6AF9
:1003880012C0DFFF1550210FD96EDA6A10C0DFFFE7
:10039800CCD00E0E1518D8A403D012C047F0C5D083
:1003A8000F0E1518D8A4C1D012C048F0BED014A0A2
:1003B80002D0128E01D0129E14A202D0128001D057
:1003C800129014A402D0128C01D0129C14A602D050
:1003D800128201D0129214A802D0128A01D0129A65
:1003E80014AA02D0128401D012940FA002D012884D
:1003F80001D012980EA202D0128601D012960FA434
:1004080002D0108E01D0109E14AE02D0108001D000
:10041800109013A002D0108C01D0109C13A202D00F
:10042800108201D0109213A402D0108A01D0109A21
:1004380013A602D0108401D010940DAA02D01088FF
:1004480001D010980EA402D0108601D010960DAEDF
:1004580002D00B8E01D00B9E13A802D00B8001D0C6
:100468000B9013AA02D00B8C01D00B9C13AC02D0BA
:100478000B8201D00B9213AE02D00B8A01D00B9ADB
:100488000FA202D00B8401D00B940DAC02D00B88C4
:1004980001D00B980EA602D00B8601D00B96060E43
:1004A800156012D015503E0FD96EDA6A12C0DFFF00
:1004B8001550300FD96EDA6A10C0DFFF1550660F7D
:1004C800D96EDA6A0BC0DFFF050E156415D00C0E65
:1004D800156012D01550310FD96EDA6A12C0DFFFDD
:1004E8001550230FD96EDA6A10C0DFFF15505A0F66
:1004F800D96EDA6A0BC0DFFF0B0E156416D00C0E2E
:100508001518D8A404D012C03DF010C02FF00F0E5B
:100518001518D8A404D012C044F010C036F01550F5
:10052800390FD96EDA6A0BC0DFFFF2900AC0F4FF08
:1005380009C0F3FF08C0DAFF07C0D9FF06C0E0FF13
:1005480005C0E8FF04C0D8FF01901000E8EF0BF0E9
:10060000007075736820627574746F6E20746F204B
:10061000736574206D6F64650020202020202020E9
:100620002020202020202020535953383000002043
:100630002020202020202020202020202020205387
:10064000595331000020202020202020202020206D
:1006500020202053595338304100002020202020F2
:1006600020202020202020202053595338304200C1
:10067000002020202020202020202020202020209A
:10068000205343414E000020202020202020202005
:1006900020202020554E4B4E4F574E00002020204A
:1006A000202020202020202020202020202020204A
:1006B000200020202047544220446973706C6179E7
:1006C000205465737400474F4449312F3830205609
:1006D0006572202573002020207777772E6C697350
:1006E000792E64657600756E6B6E6F776E204D6F38
:1006F00064757300302E38380000D388D38AD38CC9
:10070000D396FC0ED3169B8CD2AEFED70F01386B5E
:10071000896ABF0E926E396BFE0E936EF19EF00EDB
:10072000616E3A6B8B6AE00E946E3B6B95683C6B26
:100730000F0E966EF2966288628A628C628EF086E6
:10074000F18AF088F188F28EF28C1EEC0CF0010137
:10075000DB6B000EDA6FDA51290FD96EDA6A200EE0
:10076000DF6EDA51300FE16EE26ADFCFE7FFDA5178
:10077000370FD96EDA6AE7CFDFFFDA513E0FE16E4D
:10078000E26ADFCFE7FFDA4BDB2BDBBFE4D7DB51DD
:1007900004E1070EDA5DD8A0DED7DB6B000EDA6F5E
:1007A000DA51600FD96EDA6A200EDF6EDA51660F09
:1007B000E16EE26ADFCFE7FFDA4BDB2BDBBFF0D77E
:1007C000DB5104E1060EDA5DD8A0EAD7DB6B000E40
:1007D000DA6FDA51450FD96EDA6A200EDF6EDA4B26
:1007E000DB2BDBBFF6D7DB5104E1040EDA5DD8A0CA
:1007F000F0D7B90E166E010E176E2E0E186E185029
:10080000D8A4060E196EA1EC0CF0A40E166E010E03
:10081000176E2E0E186E1850D8A4060E196EA1EC85
:100820000CF08F0E166E010E176E2E0E186E1850ED
:10083000D8A4060E196EA1EC0CF07A0E166E010EFD
:10084000176E2E0E186E1850D8A4060E196EA1EC55
:100850000CF000018A6B9F6BB46BC96BDE6BF36BA2
:1008600001018E6BA36BB86BCD6B010EE9EC0CF044
:10087000070EC9EC0DF0496E48D0A00E166E176A2F
:10088000710E186E1850D8A4060E196EA1EC0CF05B
:100890004FD0A00E166E176A190E186E1850D8A4F5
:1008A000060E196EA1EC0CF043D0A00E166E176A5E
:1008B000450E186E1850D8A4060E196EA1EC0CF057
:1008C00037D0A00E166E176A5B0E186E1850D8A49B
:1008D000060E196EA1EC0CF02BD0A00E166E176A46
:1008E0002F0E186E1850D8A4060E196EA1EC0CF03D
:1008F0001FD0A00E166E176A870E186E1850D8A457
:10090000060E196EA1EC0CF013D04950000AD8B4B1
:10091000D8D7010AD8B4BDD7030AD8B4C6D7010ABC
:10092000D8B4DBD7070AD8B4A8D7010AD8A4E1D72E
:10093000050E496402D0040E496E050E4918D8A46C
:1009400002D0F29608D04950D8A404D0F296F0868E
:10095000F08803D0F286F096F09813EC0AF0050EBA
:100960004918D8A43ED0DF0E0001F96FC60EFA6F09
:10097000F40EFB6FFB51D8A4060EFC6F0CEC0DF0CF
:10098000000E1A6E000E2CEC0DF0DF0E1A6E1B6AB4
:1009900067EC0DF0010E1A6E000E2CEC0DF0B20E8D
:1009A0001A6E1A50D8A4060E1B6E67EC0DF0020EDC
:1009B0001A6E000E2CEC0DF0010E1A6E1A50D8A40F
:1009C000060E1B6E67EC0DF0030E1A6E000E2CEC7B
:1009D0000DF0D60E1A6E1A50D8A4060E1B6E67ECD8
:1009E0000DF0040E4918D8A439D0030E1A6E000E6B
:1009F0002CEC0DF0A00E1A6E1B6A67EC0DF0530E76
:100A00000001DF6F540EE06F520EE16F3A0EE26F9D
:100A10000101DB6B000EDA6F400EDA25D96E010E94
:100A2000DB21DA6EDE04D8A406D0DA51E30FD96EEA
:100A3000DA6A540E05D0DA51E30FD96EDA6A2D0E58
:100A4000DF6EDA4BDB2BDBBFE7D7DB5104E1100EA7
:100A5000DA5DD8A0E1D70001F36B7FD34904D8A4B5
:100A60001ED1200E0001E16FE1C0E0F0E0C0DFF038
:100A7000435030EC09F00001E26F425030EC09F0D5
:100A80000001E36F415030EC09F00001E46F405089
:100A900030EC09F00001E56F3F5030EC09F0000147
:100AA000E66F3E5030EC09F00001E76F200EE86F72
:100AB000200EEB6FEBC0EAF0EAC0E9F03C5030ECFE
:100AC00009F00001EC6F3B5030EC09F00001ED6FD4
:100AD0003A5030EC09F00001EE6F395030EC09F07B
:100AE0000001EF6F385030EC09F00001F06F375023
:100AF00030EC09F00001F16F200EF26FF36B200E65
:100B0000CC6FCCC0CBF0CBC0CAF0355030EC09F084
:100B10000001CD6F345030EC09F00001CE6F33503E
:100B200030EC09F00001CF6F325030EC09F00001D9
:100B3000D06F315030EC09F00001D16F305030EC03
:100B400009F00001D26F200ED36F200ED66FD6C0F1
:100B5000D5F0D5C0D4F02E5030EC09F00001D76F9D
:100B60002D5030EC09F00001D86F2C5030EC09F01A
:100B70000001D96F2B5030EC09F00001DA6F2A50D8
:100B800030EC09F00001DB6F295030EC09F0000176
:100B9000DC6F200EDD6FDE6B200EB76FB7C0B6F0D6
:100BA000B6C0B5F06B5130EC09F00001B86F6A5176
:100BB00030EC09F00001B96F695130EC09F0000127
:100BC000BA6F685130EC09F00001BB6F675130EC2F
:100BD00009F00001BC6F665130EC09F00001BD6FF7
:100BE000200EBE6F200EC16FC1C0C0F0C0C0BFF0EC
:100BF000655130EC09F00001C26F645130EC09F02E
:100C00000001C36F635130EC09F00001C46F625101
:100C100030EC09F00001C56F615130EC09F00001C2
:100C2000C66F605130EC09F00001C76F200EC86F2D
:100C3000C96B200EA26FA2C0A1F0A1C0A0F04850C5
:100C400030EC09F00001A36F475030EC09F00001CF
:100C5000A46F200EA56F465030EC09F00001A66F7E
:100C6000455030EC09F00001A76F200EA96FA9C014
:100C7000A8F0200EAC6FACC0ABF0ABC0AAF0200E59
:100C8000AD6F200EAE6F530EAF6F590EB06F530E97
:100C9000B16F380EB26F300EB36FB46B5ED2495085
:100CA000D8A449D08B0E166E650E176E010E186E05
:100CB00054EC0CF016501710D8B413D0000E1A6E66
:100CC000000E2CEC0DF08B0E1A6E1B6A67EC0DF00B
:100CD000650E166E010E176E8B0E186E196AA1EC5A
:100CE0000CF0760E166E500E176E010E186E54EC48
:100CF0000CF016501710D8B413D0010E1A6E000E57
:100D00002CEC0DF0760E1A6E1B6A67EC0DF0500E8F
:100D1000166E010E176E760E186E196AA1EC0CF0A5
:100D2000030E1A6E000E2CEC0DF0A00E1A6E1B6A4C
:100D300067EC0DF012D2020E4918D8A428D1200E6B
:100D40000001E16FE1C0E0F0E0C0DFF0435030ECC3
:100D500009F00001E26F425030EC09F00001E36F4E
:100D6000415030EC09F00001E46F405030EC09F0E4
:100D70000001E56F3F5030EC09F00001E66F3E5096
:100D800030EC09F00001E76F445030EC09F000014D
:100D9000E86F200EEB6FEBC0EAF0EAC0E9F03C50E0
:100DA00030EC09F00001EC6F3B5030EC09F0000131
:100DB000ED6F3A5030EC09F00001EE6F395030EC35
:100DC00009F00001EF6F385030EC09F00001F06FCE
:100DD000375030EC09F00001F16F3D5030EC09F074
:100DE0000001F26FF36B200ECC6FCCC0CBF0CBC008
:100DF000CAF0355030EC09F00001CD6F345030ECC2
:100E000009F00001CE6F335030EC09F00001CF6FD4
:100E1000325030EC09F00001D06F315030EC09F065
:100E20000001D16F305030EC09F00001D26F365024
:100E300030EC09F00001D36F200ED66FD6C0D5F08C
:100E4000D5C0D4F02E5030EC09F00001D76F2D50F2
:100E500030EC09F00001D86F2C5030EC09F00001A3
:100E6000D96F2B5030EC09F00001DA6F2A5030ECCA
:100E700009F00001DB6F295030EC09F00001DC6F54
:100E80002F5030EC09F00001DD6FDE6B200EB76FE4
:100E9000B7C0B6F0B6C0B5F06B5130EC09F0000148
:100EA000B86F6A5130EC09F00001B96F695130EC4C
:100EB00009F00001BA6F685130EC09F00001BB6F16
:100EC000675130EC09F00001BC6F665130EC09F05D
:100ED0000001BD6F200EBE6F200EC16FC1C0C0F0FB
:100EE000C0C0BFF0655130EC09F00001C26F645121
:100EF00030EC09F00001C36F635130EC09F00001E0
:100F0000C46F625130EC09F00001C56F615130ECE3
:100F100009F00001C66F605130EC09F00001C76FA5
:100F2000200EC86FC96B200EA26FA2C0A1F0A1C095
:100F3000A0F0485030EC09F00001A36F475030ECAE
:100F400009F00001A46F200EA56F465030EC09F0A7
:100F50000001A66F455030EC09F00001A76F200E8C
:100F6000A96FA9C0A8F0200EAC6FACC0ABF0ABC0AD
:100F7000AAF0200EAD6F530EAE6F590EAF6F530E29
:100F8000B06F380EB16F300EB26F410E85D6030EC2
:100F90004918D8A4DBD0200E0001E16FE1C0E0F0D9
:100FA000E0C0DFF0435030EC09F00001E26F425046
:100FB00030EC09F00001E36F415030EC09F0000122
:100FC000E46F405030EC09F00001E56F3F5030EC29
:100FD00009F00001E66F3E5030EC09F00001E76FC8
:100FE000200EE86F200EEB6FEBC0EAF0EAC0E9F0EC
:100FF0003C5030EC09F00001EC6F3B5030EC09F054
:101000000001ED6F3A5030EC09F00001EE6F3950FD
:1010100030EC09F00001EF6F385030EC09F00001BE
:10102000F06F375030EC09F00001F16F200EF26FD5
:10103000F36B200ECC6FCCC0CBF0CBC0CAF03550D8
:1010400030EC09F00001CD6F345030EC09F00001B4
:10105000CE6F335030EC09F00001CF6F325030ECDE
:1010600009F00001D06F315030EC09F00001D16F70
:10107000305030EC09F00001D26F200ED36F200EFB
:10108000D66FD6C0D5F0D5C0D4F02E5030EC09F0D4
:101090000001D76F2D5030EC09F00001D86F2C50B3
:1010A00030EC09F00001D96F2B5030EC09F0000151
:1010B000DA6F2A5030EC09F00001DB6F295030EC78
:1010C00009F00001DC6F200EDD6FDE6BB50E166ED1
:1010D000176A9D0E186E1850D8A4060E196EA1EC52
:1010E0000CF0200E0001A26FA2C0A1F0A1C0A0F0E0
:1010F000485030EC09F00001A36F475030EC09F084
:101100000001A46F200EA56F465030EC09F00001DD
:10111000A66F455030EC09F00001A76F200EA96FB3
:10112000A9C0A8F0200EAC6FACC0ABF0ABC0AAF069
:10113000200EAD6F200EAE6F200EAF6F530EB06F4E
:10114000590EB16F530EB26F310EA6D5DF0E0001EE
:10115000F96FE60EFA6F0CEC0DF04950D8B4ADEF14
:1011600004F0DF0E166EB90E176E010E186E54ECF9
:101170000CF016501710D8B413D0B90E166E010E1D
:10118000176EDF0E186E196AA1EC0CF0000E1A6EC5
:10119000000E2CEC0DF0DF0E1A6E1B6A67EC0DF0E2
:1011A000CA0E166EA40E176E010E186E54EC0CF0DB
:1011B00016501710D8B413D0A40E166E010E176E69
:1011C000CA0E186E196AA1EC0CF0010E1A6E000E10
:1011D0002CEC0DF0CA0E1A6E1B6A67EC0DF0B50E02
:1011E000166E8F0E176E010E186E54EC0CF0165022
:1011F0001710D8B413D08F0E166E010E176EB50EE1
:10120000186E196AA1EC0CF0020E1A6E000E2CEC8E
:101210000DF0B50E1A6E1B6A67EC0DF0A00E166E7F
:101220007A0E176E010E186E54EC0CF01650171053
:10123000D8B4ADEF04F07A0E166E010E176EA00E44
:10124000186E196AA1EC0CF0030E1A6E000E2CEC4D
:101250000DF0A00E1A6E1B6A67EC0DF0ADEF04F0F6
:10126000166E53D0200E4FD02B0E4DD02D0E4BD0DE
:10127000300E49D0310E47D0320E45D0330E43D018
:10128000340E41D0350E3FD0360E3DD0370E3BD018
:10129000380E39D0390E37D0410E35D0420E33D00A
:1012A000430E31D0440E2FD0450E2DD0460E2BD0FC
:1012B000470E29D0480E27D0490E25D04A0E23D0FC
:1012C0004B0E21D04C0E1FD04D0E1DD04E0E1BD0FC
:1012D000500E19D0520E17D0540E15D0550E13D0F3
:1012E000560E11D0570E0FD0580E0DD0590E0BD0F0
:1012F000610E09D0620E07D0630E05D0640E03D0D4
:10130000650E01D03F0E176E8CD01650000AD8B46F
:10131000A9D7080AD8B4AED7180AD8B4A7D7050AEF
:10132000D8B4EAD7020AD8B4DBD70F0AD8B49CD70E
:101330003E0AD8B4C7D7080AD8B4D2D71C0AD8B442
:10134000D7D7040AD8B4DCD70A0AD8B4B9D76E0AFA
:10135000D8B4D0D7070AD8B493D7020AD8B4C6D71E
:101360000B0AD8B4C1D7030AD8B4B4D73C0AD8B44E
:10137000A5D7040AD8B4B2D7080AD8B4B3D71F0A7D
:10138000D8B4A4D7050AD8B495D7030AD8B47CD763
:101390000B0AD8B4A9D7F50AD8B49ED7020AD8B494
:1013A0008BD71C0AD8B4AAD7320AD8B493D7020A6A
:1013B000D8B476D7150AD8B45FD7070AD8B476D789
:1013C000010AD8B485D7030AD8B46ED7770AD8B43F
:1013D0005DD70A0AD8B466D7180AD8B44FD7060A18
:1013E000D8B458D7030AD8B44DD7010AD8B452D7C5
:1013F0000C0AD8B453D73E0AD8B468D7030AD8B475
:1014000057D7010AD8B434D70A0AD8B45DD7180A16
:10141000D8B442D7030AD8B437D7010AD8B438D7DA
:1014200071D717501200000E84B6010E1E6E1E50AA
:10143000D8A4CDD00001FE05D8A4C9D04928496E52
:10144000050E496401D0496A49C016F0070EB3EC95
:101450000DF0010EE9EC0CF0DF0E166E176A2E0E81
:10146000186E1850D8A4060E196EA1EC0CF0CA0E16
:10147000166E176A2E0E186E1850D8A4060E196E26
:10148000A1EC0CF0B50E166E176A2E0E186E1850E1
:10149000D8A4060E196EA1EC0CF0B90E166E010E52
:1014A000176E2E0E186E1850D8A4060E196EA1ECE9
:1014B0000CF0A40E166E010E176E2E0E186E18503C
:1014C000D8A4060E196EA1EC0CF08F0E166E010E4C
:1014D000176E2E0E186E1850D8A4060E196EA1ECB9
:1014E0000CF07A0E166E010E176E2E0E186E185036
:1014F000D8A4060E196EA1EC0CF048D0A00E166E02
:10150000176A710E186E1850D8A4060E196EA1EC49
:101510000CF04FD0A00E166E176A190E186E1850E8
:10152000D8A4060E196EA1EC0CF043D0A00E166ED6
:10153000176A450E186E1850D8A4060E196EA1EC45
:101540000CF037D0A00E166E176A5B0E186E18508E
:10155000D8A4060E196EA1EC0CF02BD0A00E166EBE
:10156000176A2F0E186E1850D8A4060E196EA1EC2B
:101570000CF01FD0A00E166E176A870E186E18504A
:10158000D8A4060E196EA1EC0CF013D04950000A35
:10159000D8B4D8D7010AD8B4BDD7030AD8B4C6D7AF
:1015A000010AD8B4DBD7070AD8B4A8D7010AD8A44F
:1015B000E1D7050E4918D8B403D04950D8A404D0B7
:1015C000F296F086F08803D0F286F096F0981EC06E
:1015D000FEF012002150D96EDA6ADFCFF6FF060E58
:1015E000F76E0800F550250AD8A498D02150D96E7E
:1015F000DA6ADF2A00016D6B000E6C6F6CC072F04E
:101600006E696F69256A2150D96EDA6ADFCFF6FFFD
:10161000060EF76E0800F550730AD8A407D02150C3
:10162000D96EDA6ADF2A010E256E32D02150D96ECA
:10163000DA6ADFCFF6FF060EF76E0800F5506C0A87
:10164000D8A426D02150D96EDA6ADF50246E010E5C
:10165000242624C0F6FF060EF76E0800F5506C0A2B
:10166000D8A416D02150D96EDA6ADF50246E020E4B
:10167000242624C0F6FF060EF76E0800F550730A04
:10168000D8A406D02150D96EDA6A030EDF26CBD754
:101690002550D8B43ED022C0D9FF23C0DAFF020EB5
:1016A000DF26DF5CD96EDA6ADECF26F0DECF27F0E8
:1016B0001CD026C0F6FF27C0F7FFF86A050EF764B6
:1016C00003D00800F55005D0F6CFE1FFF7CFE2FFD9
:1016D000E750246E2450166E176A1FC018F020C001
:1016E00019F0A0EC0BF0264A272A26C0F6FF27C0E7
:1016F000F7FFF86A050EF76403D00800F55005D02F
:10170000F6CFE1FFF7CFE2FFE7500009D8B41200AF
:10171000D0D72150D96EDA6ADF2A12002150D96E53
:10172000DA6ADFCFF6FF060EF76E0800F550166E88
:10173000176A1FC018F020C019F0A0EC0BF0E9D711
:1017400018501910D8B404D018501910D8A404D0C7
:101750001650D7EC0DF0120020EE09F01850D926E3
:101760001950DA22DE50DE10D8B416D020EE09F07F
:101770001850D9261950DA2210EE02F01850E1263E
:101780001950E222DE50E65CE650800A1E6EDE5002
:10179000800A1E58D8B0120020EE02F01850D92648
:1017A0001950DA22DF501A6E18C0D9FF19C0DAFFBB
:1017B000DF501A24D96EDA6A16C0DFFF20EE02F07D
:1017C0001850D9261950DA22DE2A000EDD22120026
:1017D000B00EF66E1B0EF76E000EF86E0900F5CF18
:1017E000FEF003EE00F011EE00F0EE6AE550E1507D
:1017F000FCE1E250FAE102EE00F011EE00F0EE6AD8
:10180000E550E150FCE1E250FAE101EE00F0CE0ECD
:10181000EE6AE806FDE100EE60F0940EEE6AE8067E
:10182000FDE100EE29F0230EEE6AE806FDE10190ED
:101830000192000EF86E00017DEF03F08A90809C0B
:101840008290960E7BEC0CF0300E83EC0DF0050EC2
:10185000E82EFED70000D1EC0DF0290E7BEC0CF049
:10186000D1EC0DF0010E7BEC0CF0D1EC0DF09BEC0B
:101870000DF0200E83EC0DF0050EE82EFED70000D3
:10188000D1EC0DF09BEC0DF0010EE9EC0CF0280E04
:10189000E9EC0CF0080EE9EC0CF0060EE9EC0CF0AB
:1018A0000C0EE9EC0CF0120003D0162A174A182A85
:1018B00017C0D9FF18C0DAFF1650E16EE26ADE5099
:1018C000E618D8A406D01650D96EDA6ADF50D8A42C
:1018D000ECD71650D96EDA6ADF50196E17C0D9FFEF
:1018E00018C0DAFFDF501A6E1A50195C166E176AAC
:1018F000D8A017061200196E1B6A000E1A6E13D0BC
:101900001D6A000E1C6E350EE82EFED700001C4A24
:101910001D2A1DBEF8D71D5004E10A0E1C5CD8A07C
:10192000F2D71A4A1B2A1950166E176A16501A5CFB
:101930001B50800A186E1750800A1858D8B0120031
:10194000DFD716C01CF017C01DF018501A6E1950C2
:101950001B6E184A192A1AC0F6FF1BC0F7FFF86A57
:101960001CC0D9FF1DC0DAFF1C4A1D2A050EF764F2
:1019700003D00800F55005D0F6CFE1FFF7CFE2FF26
:10198000E750DF6EDF50D8B41200DFD7196E9BEC42
:101990000DF01950F00B186E185083EC0DF0150E69
:1019A000E82EFED70000809C8A800A0EE82EFED723
:1019B00000D0D1EC0DF0193A1950F00B186E1850F8
:1019C00083EC0DF0150EE82EFED70000D1EC0DF0E3
:1019D0001200196E9BEC0DF01950F00B186E185098
:1019E00083EC0DF0150EE82EFED70000809C8A9047
:1019F0000A0EE82EFED700D0D1EC0DF0193A19509E
:101A0000F00B186E185083EC0DF0150EE82EFED773
:101A10000000D1EC0DF01200FB0E0101CE6FF9C0F9
:101A2000CFF1D26B000ED16FD96B000ED86FCF0EF5
:101A30000001F46F010EF56FFAC0F6F0CE0EF76FED
:101A4000010EF86F4AEC0DF00001F9510101D125AA
:101A5000D96EDA6ADF6A12001B6E130E1B6408D09F
:101A600012001B8C12D0140E01D0540E1B260DD068
:101A70001A50000AD8B409D0010AD8B4F2D7030A20
:101A8000D8B4F1D7010AD8B4F0D71B8E1B50E9ECBB
:101A90000CF01200F6C028F00CD0F4C01FF0F5C016
:101AA00020F0280E216EF7C022F0F8C023F0EAECF7
:101AB0000AF028C0F6FF060EF76E0800F550000980
:101AC000D8A4EBD70001F56B000EF46F12001AC01A
:101AD000F6FF1BC0F7FFF86A050EF76403D0080095
:101AE000F55005D0F6CFE1FFF7CFE2FFE7501C6ECF
:101AF00006D01C50C6EC0CF01A4A1B2AE8D71C5022
:101B0000D8B41200F6D7166E16C017F017A802D078
:101B1000828201D0829217AA02D0828401D082945C
:101B200017AC02D0828601D0829617AE02D082888E
:101B300001D08298120094888A90808CD1EC0DF0AC
:101B4000350EE82EFED70000000E8BB8010E166E83
:101B5000D1EC0DF01650D8A4EED7809C9498500E7E
:101B6000E82EFED71200176E01D00000A6B2FDD7F6
:101B7000A19817C0A9FF16C0A8FFA69EA69CA68480
:101B8000F29E550EA76EAA0EA76EA682F28EA6949E
:101B90001200166E16C0A9FFA69EA69CA680A8508D
:101BA00012008280100EE82EFED7829012001200E2
:011BB0000133
:020000040020DA
:08000000FFFFFFFFFFFFFFFF00
:020000040030CA
:0E000000FF381E3CFF3581FF0FC00FE00F40A0
:00000001FF
